:020000040000FA
:0600000007309F00F82903
:08000800BC00030EBD008B1AC1
:100010002B280B1A1B283D0E8300BC0E3C0E09003A
:10002000810183166400883081008312851490302A
:100030008B00BB0108008B100C30B700B70B1E28DB
:1000400006180B28AD30810020308B000230BB0039
:100050000830B7000B280B113B193E28B7080319CD
:100060003728060CB80CB703AD3081000B28061CEE
:1000700058280130BB003808B9005828BB19582847
:10008000B70803195028BA0C031C4928000085142E
:100090004C28851000000000B703B53081000B2804
:1000A0000000000000008514BB15A83081000B285B
:1000B00010308B000130BB050B2885100630BB00CB
:1000C0000000B5308100A0308B000830B700080078
:1000D00080213B1C68283B1008005D208021BB1854
:1000E0006E2808008207482A532A5F2A6B2A772A3B
:1000F000BA2AC72ACF2AD72A5334653472344434F3
:10010000443453342034763431342E343034003493
:100110004634723465347134003453347434613489
:1001200072347434003445346E34643400345334DF
:1001300074346534703400345334633461346E3451
:100140000034533468346F347734003455347034A9
:10015000203428346F34723420343E34293400344F
:1001600044346F3477346E34203428346F3472342E
:1001700020343C3429340034483465346C347034D1
:100180000034BF09C009C109C209BF0A031DCF2835
:10019000C00A031DCF28C10A031DCF28C20A2308A5
:1001A0004207A300220841070318E820A200210803
:1001B00040070318E520A10020083F070318E220AC
:1001C000A0000800A10A031D0800A20A031D0800E0
:1001D000A30A08003030BE0203190800CF20BE0B6E
:1001E000EE2808004308BE00C2019830C1009630D6
:1001F000C0008030BF00EA204408BE000F30C100BC
:100200004230C0004030BF00EA204508BE00013047
:10021000C1008630C000A030BF00EA204608BE0002
:10022000C1012730C0001030BF00EA204708BE00DF
:100230000330C000E830BF00EA204808BE00C0011B
:100240006430BF00EA204908BE000A30BF00EA203F
:100250004A08BE000130BF00EA20080030308000AC
:10026000C120A31B3629800ACF203129C1200800D4
:1002700043308400C2019830C1009630C000803005
:10028000BF002E21840AC2010F30C1004230C000DD
:100290004030BF002E21840AC2010130C1008630E7
:1002A000C000A030BF002E21840AC201C101273046
:1002B000C0001030BF002E21840AC201C1010330EA
:1002C000C000E830BF002E21840AC201C101C00174
:1002D0006430BF002E21840AC201C101C0010A306E
:1002E000BF002E21840AC201C101C0010130BF003C
:1002F0002E210800A001A101A201A301F220080003
:1003000008003B1C81293B103908BA006D203908D0
:100310000800A401A501A601A701A8012030A90099
:100320002C08B0002D08B1002E08B2002F08B30031
:100330000310301CB2292008A507031CA429A60F0E
:10034000A429A70FA429A80A2108A607031CAB29E2
:10035000A70FAB29A80A2208A707031CB029A80ADF
:100360002308A807A80CA70CA60CA50CA40CB30C7A
:10037000B20CB10CB00CA90B9829A8010130A8004F
:100380000800243084000008AB000830AA00AB0C41
:10039000031CCE29861506150611D12986110615CE
:1003A0000611AA0BC729840A29300402031CC32999
:1003B000861786130800E021E021E021E0210800F3
:1003C000E321E3210800FF30B400F1298030B400BC
:1003D000F1294030B400F1292030B400F129103067
:1003E000B400FF30B500B50BF329B40BF1290800B8
:1003F0008B0183168113F53085000130860083124E
:100400000030A4000030A5000030A6000030A70096
:100410000030A800C1211730AF00DC30AE006530DD
:10042000AD00DE30AC00203035238921C121C1214F
:100430001020E321F422F4220930FB22F422D922F5
:10044000F4223E30BA006D202030BA006D206820C2
:1004500039083E3C031D2F2A4730B900352A390898
:100460003C3C031D352A4830B9009F3E031C3A2A04
:100470002030B90241303902031C462A4A30390281
:100480000318462A413039027220202AD722202A16
:100490001530FB22052369237A218921C1213023CC
:1004A000F4220C2308001A30FB22052369237A2149
:1004B000203084000430CC23F4220C2308002030A8
:1004C000FB22052369237A21203084000830CC23C5
:1004D000F4220C2308002430FB22052369237A210F
:1004E000203084000C30CC23F4220C230800293067
:1004F000FB220523F422203039233F304123892178
:10050000C1213023C120A31FA32A45230D30BA00E7
:100510006D20E621203035233F303D23CF203F3072
:100520004123C120A31F992A1E233B1C852A682032
:10053000B72A203041238921C121302345230D30A2
:10054000BA006D20B72A45230D30BA006D20E62190
:10055000203035233F303D23C1203F304123C1208F
:10056000A31B992A27233B1CA32A6820B72AF4221D
:100570000C2308002E30FB22F4224523F4224E23C4
:10058000F4225723F4226023F4220C230800333092
:10059000FB22F4221E234523F4220C2308003D30C5
:1005A000FB22F42227234523F4220C2308004930A0
:1005B000FB224130BE001530B600F4223E08BA00DE
:1005C0006D200523EB22BE0A4A303E02031DDD2AC0
:1005D000F4220C2308003608B60A7220FF390319EA
:1005E0000800BA006D20EB2A0D30BA006D200A30E9
:1005F000BA006D200800B60036087220FF390319D2
:100600000800BA006D20B60AFC2A3A30BA006D2004
:100610002030BA006D2008006F30BA006D206B30BA
:10062000BA006D20F42208002030BA006D20483056
:10063000BA006D207A30BA006D20080020303523D2
:100640003F303D23CF208921C121302308002030B5
:1006500035233F303D23C1208921C12130230800AB
:10066000203084000030CC23080084000030BD23FB
:10067000080084000430BD23080084000C30BD2332
:10068000080084000830BD2308001530FB22052334
:10069000203035233821B223142308001A30FB22DE
:1006A0000523203039233821B223142308002030B9
:1006B000FB220523203041233821B22314230800D4
:1006C0002430FB22052320303D233821B22314237C
:1006D00008000830B600433084008001840AB60B5D
:1006E0006D2B0830B6004330840068200830390292
:1006F0000319902B0D30390203199F2B303039022A
:10070000031C752B3A3039020318752BB6080319F0
:10071000752B39088000BA006D20840AB603752B4A
:10072000B619752BB60A840380013908BA006D200A
:100730002030BA006D203908BA006D20752BB6083C
:1007400003190800493084000730BE000008840AFD
:10075000800084038403BE0BA62B3030C300B60B8D
:10076000A22B08000830B600433084000008BA000D
:100770006D20840AB60BB62B080083169B008312EB
:100780000430B60083161C141A089B0A8000840AE1
:100790008312B60BC22B080083169B008312043011
:1007A000B6008B13831600089A009C011C15553067
:1007B0009D00AA309D009C149C18DC2B9C139B0A66
:0E07C00083128C13840AB60BD22B8B17080001
:02400E00093F68
:1042000028000100D600000080009F00D5000000BB
:10421000B000F600DA0000006400000000000000BA
:00000001FF
